:020000040000FA
:1000000098EF22F0F76A140FF66E000EF72209003F
:10001000F5501200280C0106F76A280FF66E000E44
:10002000F7220900F5501200000000000000005FF8
:1000300000000007000700147F147F14242A7F2A81
:10004000122313086462364955225000050300004C
:10005000001C2241000041221C0014083E08140824
:10006000083E080800503000000808080808006032
:1000700060000020100804023E5149453E00427FC6
:10008000400042615149462141454B311814127FCD
:100090001027454545393C4A494930017109050356
:1000A0003649494936064949291E003636000000BE
:1000B0005636000008142241001414141414004190
:1000C0002214080201510906324979413E7E11117C
:1000D000117E7F494949363E414141227F414122BB
:1000E0001C7F494949417F090909013E4149497A33
:1000F0007F0808087F00417F41002040413F017F89
:10010000081422417F404040407F020C027F7F0460
:1001100008107F3E4141413EF76A280FF66E010EFE
:10012000F7220900F55012007F090909063E4151E6
:10013000215E7F09192946464949493101017F015C
:10014000013F4040403F1F2040201F3F4038403F7C
:100150006314081463070870080761514945430098
:100160007F41410002040810200041417F00040249
:100170000102044040404040000102040020545469
:1001800054787F48444438384444442038444448F0
:100190007F3854545418087E0901020C5252523EC2
:1001A0007F0804047800447D40002040443D007FE7
:1001B0001028440000417F40007C041804787C082B
:1001C00004047838444444387C1414140808141483
:1001D000187C7C080404084854545420043F4440CC
:1001E000203C4040207C1C2040201C3C4030403CB7
:1001F00044281028440C5050503C4464544C440053
:100200000836410000007F00000041360800100859
:100210000810087846414678F76A280FF66E020EF5
:10022000F7220900F55012004272696768746E6522
:1002300073730000F76A440FF66E020EF72209008E
:10024000F550120041646A7573740000F76A5C0F20
:10025000F66E020EF7220900F5501200546563682D
:1002600044657369676E2E626500F76A7A0FF66EF1
:10027000020EF7220900F5501200566F703D20253E
:1002800075200000F76A940FF66E020EF72209003F
:10029000F550120000020001800040002000100014
:1002A0000800040002000100DC026E01B7008702B2
:1002B0009F03130355037603BB010102DC03EE0128
:1002C000F700A7028F031B03F76AD80FF66E020E22
:1002D000F7220900F55012002D2D2D2D2D2D2D2D3D
:1002E0000000F76AF20FF66E020EF7220900F550D1
:1002F00012002020202020506F70204D75736963FC
:100300002020202020200000F76A180FF66E030E30
:10031000F7220900F550120020202020204D4F52D6
:10032000204D757369632020202020200000F76A8B
:100330003E0FF66E030EF7220900F5501200202042
:10034000202020204C6569737572652020202020B4
:1003500020200000F76A640FF66E030EF7220900F2
:10036000F550120020536572696F757320436C61FC
:1003700073736963616C20200000F76A8A0FF66E60
:10038000030EF7220900F550120020202020202023
:1003900020204E6577732020202020202020000080
:1003A000F76AB00FF66E030EF7220900F55012003F
:1003B000202043757272656E7420416666616972B1
:1003C000732020200000F76AD60FF66E030EF72286
:1003D0000900F550120020202020496E666F726DD2
:1003E0006174696F6E20202020200000F76AFC0FE6
:1003F000F66E030EF7220900F5501200202020208F
:1004000020202053706F7274202020202020202074
:100410000000F76A220FF66E040EF7220900F5506D
:1004200012002020202020456475636174696F6E7E
:100430002020202020200000F76A480FF66E040ECE
:10044000F7220900F550120020202020202020440F
:1004500072616D6120202020202020200000F76A9A
:100460006E0FF66E040EF7220900F55012002020E0
:100470002020202043756C74757265202020202078
:1004800020200000F76A940FF66E040EF722090090
:10049000F5501200202020202020536369656E63F0
:1004A00065202020202020200000F76ABA0FF66E79
:1004B000040EF7220900F5501200202020202020F1
:1004C00056617269656420202020202020200000D1
:1004D000F76AE00FF66E040EF7220900F5501200DD
:1004E00020202020526F636B204D7573696320209C
:1004F000202020200000F76A060FF66E050EF72276
:100500000900F550120020204C6967687420436C84
:100510006173736963616C2020200000F76A2C0FFF
:10052000F66E050EF7220900F5501200202020205B
:100530004F74686572204D757369632020202020F8
:100540000000F76A520FF66E050EF7220900F5500B
:1005500012002020202020205765617468657220D9
:100560002020202020200000F76A780FF66E050E6C
:10057000F7220900F5501200202020202020466993
:100580006E616E6365202020202020200000F76A25
:100590009E0FF66E050EF7220900F5501200436813
:1005A000696C6472656E27732050726F6772616D3B
:1005B00073200000F76AC40FF66E050EF7220900DB
:1005C000F5501200202020536F6369616C20416652
:1005D00066616972732020200000F76AEA0FF66EE8
:1005E000050EF7220900F5501200202020202020BF
:1005F00052656C6967696F6E202020202020000002
:10060000F76A100FF66E060EF7220900F550120079
:1006100020202020202050686F6E6520496E202009
:10062000202020200000F76A360FF66E060EF72213
:100630000900F55012002020202020202054726153
:1006400076656C202020202020200000F76A5C0FB7
:10065000F66E060EF7220900F55012002020202029
:10066000204A617A7A204D7573696320202020200A
:100670000000F76A820FF66E060EF7220900F550A9
:100680001200202020436F756E747279204D7573AF
:100690006963202020200000F76AA80FF66E060E7E
:1006A000F7220900F55012002020204E6174696F76
:1006B0006E616C204D757369632020200000F76A1D
:1006C000CE0FF66E060EF7220900F550120020201C
:1006D00020204F6C64696573204D75736963202019
:1006E00020200000F76AF40FF66E060EF7220900CC
:1006F000F55012002020202020466F6C6B204D7595
:1007000073696320202020200000F76A1A0FF66E1C
:10071000070EF7220900F550120020202020446F18
:1007200063756D656E746172792020202020000051
:10073000F76A400FF66E070EF7220900F550120017
:100740002020202020416C61726D2054657374203C
:10075000202020200000F76A660FF66E070EF722B1
:100760000900F550120020202020202020416C613B
:10077000726D20202020202020200000F76A8C0F9E
:10078000F66E070EF7220900F550120043545F4D34
:100790004A443D20256C75200A0D0000F76AAC0F15
:1007A000F66E070EF7220900F55012004D6F00009B
:1007B000F76AC00FF66E070EF7220900F550120017
:1007C00054750000F76AD40FF66E070EF722090081
:1007D000F550120057650000F76AE80FF66E070E35
:1007E000F7220900F550120054680000F76AFC0F68
:1007F000F66E070EF7220900F5501200467200004F
:10080000F76A100FF66E080EF7220900F550120075
:1008100053610000F76A240FF66E080EF7220900F4
:10082000F550120053750000F76A380FF66E080E87
:10083000F7220900F55012004A616E00F76A4C0F6A
:10084000F66E080EF7220900F550120046656200A8
:10085000F76A600FF66E080EF7220900F5501200D5
:100860004D617200F76A740FF66E080EF7220900E8
:10087000F550120041707200F76A880FF66E080E8C
:10088000F7220900F55012004D617900F76A9C0FBC
:10089000F66E080EF7220900F55012004A756E0038
:1008A000F76AB00FF66E080EF7220900F550120035
:1008B0004A756C00F76AC40FF66E080EF72209003D
:1008C000F550120041756700F76AD80FF66E080EF2
:1008D000F7220900F550120053657000F76AEC0F1B
:1008E000F66E080EF7220900F55012004F637400EF
:1008F000F76A000FF66E090EF7220900F550120094
:100900004E6F7600F76A140FF66E090EF722090093
:10091000F550120044656300F76A280FF66E090E61
:10092000F7220900F5501200626C616E6B5F64691A
:1009300073706C617973212121200A0D0000F76A20
:100940004E0FF66E090EF7220900F55012002054E2
:1009500050200000F76A640FF66E090EF7220900B6
:10096000F5501200202020202020202020202020B0
:10097000202020200000F76A860FF66E090EF7226D
:100980000900F5501200200A0A0D0000F76A9C0FBA
:10099000F66E090EF7220900F550120020202020E3
:1009A0000000F76AB20FF66E090EF7220900F55043
:1009B0001200202020202020202020202020202065
:1009C0002000F76AD20FF66E090EF7220900F550E3
:1009D0001200202020202000F76AE80FF66E090E92
:1009E000F7220900F55012002A2020202000F76A83
:1009F000FE0FF66E090EF7220900F55012002A2AA2
:100A000020202000F76A140FF66E0A0EF722090064
:100A1000F55012002A2A2A202000F76A2A0FF66EC3
:100A20000A0EF7220900F55012002A2A2A2A20006D
:100A3000F76A400FF66E0A0EF7220900F550120011
:100A40002A2A2A2A2A00F76A560FF66E0A0EF72279
:100A50000900F55012002020202020202020000036
:100A6000F76A700FF66E0A0EF7220900F5501200B1
:100A70002020202020202020202020202020202076
:100A80002020202020202020202020202020202066
:100A90002020202020202020202020202020202056
:100AA0002020202020202020202020202020202046
:100AB0000000F76AC20FF66E0A0EF7220900F55021
:100AC0001200202020202020202020202020202054
:100AD0002020202020200000F76AE80FF66E0A0E82
:100AE000F7220900F5501200303231202D205244F7
:100AF00053204465636F646572200A0D0000F76A35
:100B00000E0FF66E0B0EF7220900F5501200202092
:100B1000524453204465636F646572200000F76A95
:100B20002E0FF66E0B0EF7220900F55012005465D9
:100B3000636844657369676E2E6265200000F76A1A
:100B40004E0FF66E0B0EF7220900F5501200202012
:100B5000303231202D20524453204465636F646548
:100B600072200000F76A740FF66E0B0EF722090070
:100B7000F550120020207777772E746563686465DE
:100B80007369676E2E6265200000F76A9A0FF66E31
:100B90000B0EF7220900F5501200696E6974204FA0
:100BA0004B200A0D0000020EEA6EDA0EE96EEF50DD
:100BB0000DE0060E016E006A002EFED7012EFBD757
:100BC0007B0E006E002EFED7EF2EF3D7000C130E17
:100BD0000201CE6FCB5302E1829403D0CB2D01D022
:100BE0008296080ECD6FCD531FE08292010ECD5D2F
:100BF000CF6FCEC200F0CF51016E04E0D89000322A
:100C0000012EFCD700B002D0829001D08280020E6B
:100C1000DA6F0001C8DF8282020E0201DA6F000182
:100C2000C2DF0201CD07DFD7080ECD6FCD531FE025
:100C30008292010ECD5DCF6FCCC200F0CF51016E1C
:100C400004E0D8900032012EFCD700B002D0829090
:100C500001D08280020EDA6F0001A5DF8282020ECF
:100C60000201DA6F00019FDF0201CD07DFD7829218
:100C7000828482860001000CF2CFCAF2F29EA96A39
:100C8000A69CA69EA680A8500201CABFF28E0001B3
:100C9000CF6FCF517F0815E3A00ECF6FA96AA86E62
:100CA000A69CA69EA684F2CF00F0F29E0F01550EE0
:100CB000A76EAA0EA76EA682A6B2FED7A694005073
:100CC000F2120001E8EF24F0080E0201DC6FDC53A1
:100CD0000CE0839ADB51800B02E1839801D083887A
:100CE000838AD890DB37DC07F2D70001000C8392AF
:100CF0008396D3C2DBF2E8DF8386000C0201D15178
:100D0000070B4009D26FD36F0001F1DF0201D05110
:100D10007F0B8009D26FD36F0001E9DF000C838263
:100D20008396DAC2DBF2D0DF8386000C0201D06B3F
:100D3000D16B0001E3DF010ED46FF80ED36FD353F4
:100D400002E1D45309E00201DA6B0001E8DFD3517C
:100D5000D8B4D407D307F3D7CFEF06F083828386C6
:100D600083940A0E0201DA6F00011DDF8384210ED5
:100D70000201D36F0001BBDFCFC0D3F2B8DF130E87
:100D80000201D36F0001B3DF200E0201D36F000117
:100D9000AEDF090E0201D36F0001A9DFC7D7080E2D
:100DA0000201D36F0001A3DF0C0E0201D36F00011B
:100DB0009EDF000CD251C70803E1800ED26FE2D053
:100DC000D251FC0803E1810ED26FDCD0D251E90888
:100DD00003E1820ED26FD6D0D251E20803E1830E36
:100DE000D26FD0D0D251E40803E1840ED26FCAD0C2
:100DF000D251E00803E1850ED26FC4D0D251E5088C
:100E000003E1860ED26FBED0D251E70803E1870E10
:100E1000D26FB8D0D251EA0803E1880ED26FB2D0B7
:100E2000D251EB0803E1890ED26FACD0D251E80861
:100E300003E18A0ED26FA6D0D251EF0803E18B0EE8
:100E4000D26FA0D0D251EE0803E18C0ED26F9AD0AF
:100E5000D251EC0803E18D0ED26F94D0D251C40868
:100E600003E18E0ED26F8ED0D251C50803E18F0EF2
:100E7000D26F88D0D251C90803E1900ED26F82D0D0
:100E8000D251E60803E1910ED26F7CD0D251C60850
:100E900003E1920ED26F76D0D251F40803E1930EA3
:100EA000D26F70D0D251F60803E1940ED26F6AD09F
:100EB000D251F20803E1950ED26F64D0D251FB08F3
:100EC00003E1960ED26F5ED0D251F90803E1970E7E
:100ED000D26F58D0D23D03D0980ED26F53D0D2519A
:100EE000D60803E1990ED26F4DD0D251DC0803E150
:100EF0009A0ED26F47D0D251F80803E19B0ED26F01
:100F000041D0D251A30803E19C0ED26F3BD0D25105
:100F1000D80803E19D0ED26F35D0D251D70803E136
:100F20009E0ED26F2FD0D251830803E19F0ED26F55
:100F300029D0D251E10803E1A00ED26F23D0D251C3
:100F4000ED0803E1A10ED26F1DD0D251F30803E1E9
:100F5000A20ED26F17D0D251FA0803E1A30ED26FBE
:100F600011D0D251F10803E1A40ED26F0BD0D251AF
:100F7000D10803E1A50ED26F05D0D251DF0802E1FE
:100F8000A60ED26FE7EF07F083828396080E020168
:100F9000DB6FDB5310E0839A030E006E002EFED74A
:100FA000DA51010B02E1839801D08388838AD890BB
:100FB000DA33DB07EED783860001000CD2511F081D
:100FC00002E386D004D0D2517F0801E2F3D6D25199
:100FD0001F0801E37DD0D251A60801E279D0D06B81
:100FE000D051040869E3D2514F081EE3D251E00FFB
:100FF000050DF350EA6BE96FD051E9250201DA6F74
:10100000000E0001EA210201DB6F036EDA51F2CF1C
:10101000DCF2F29E00010CEC00F00201DCBFF28E6B
:10102000E8CFD1F03ED00001D2517F081EE3D2516B
:10103000B00F050DF350EA6BE96FD051E9250201BD
:10104000DA6F000E0001EA210201DB6F036EDA5154
:10105000F2CFDCF2F29E00018CEC00F00201DCBF6A
:10106000F28EE8CFD1F01DD00001D251A60818E3CE
:10107000D251800F050DF350EA6BE96FD051E9258D
:101080000201DA6F000E0001EA210201DB6F0C0E93
:10109000DA25E96E000EDB21EA6EEFCFD1F0000118
:1010A00002010BA203D0FF0E0001D11BD1C0DAF266
:1010B000000135DED02B94D70BB205D00201DA6BDC
:1010C000000162DF05D0FF0E0201DA6F00015CDF74
:1010D0006DEF08F0D9C2D2F071D7000C0201D351E4
:1010E000016AD25D03E2D2C200F00CD0006A080EA1
:1010F000D46FD2370036D351005CD8B0006E0136C1
:10110000D42FF7D70001000C0150CBC2D2F2640EED
:101110000201D36F0001E2DF00C0CBF20150300EBC
:1011200008E10201CCA30ED0CCB70CD0CCB9200E74
:1011300004D00201CC97CC99CC81012601509EA805
:10114000FED7AD6ECBC2D2F20A0ED36F0001C6DF5E
:1011500000C0CBF20150300E08E10201CCB70BD039
:10116000CCA109D0CCB9200E0001012601509EA8C7
:10117000FED7AD6E0201300ECB27CB519EA8FED715
:10118000AD6E0001000C1E0E0201D06F010ED16F7A
:101190000001B4DD4C0E0201D96F00019BDF430E4C
:1011A0000201D96F000196DF440E0201D96F0001E0
:1011B00091DF0C0E0201D06F020ED16F00019EDD97
:1011C0000201CA6BCA5100010CEC01F00201CA2BEA
:1011D000006ED96F00017EDF0A0E0201CA5DF2E1E6
:1011E000180ED06F030ED16F000188DD0201CA6BAB
:1011F000CA5100011AEC01F00201CA2B006ED96F2E
:10120000000168DF060E0201CA5DF2E1030ED06F35
:10121000050ED16F000172DD0201CA6BCA510001D7
:1012200026EC01F00201CA2B006ED96F000152DFDB
:101230000D0E0201CA5DF2E180A031D00001CF3D68
:1012400003D002012CD00001010ECF27C80E0201ED
:10125000DA6F0001A8DC210E0201D36F000147DD27
:10126000CFC0D3F244DD0201CA6BCA51000135EC94
:1012700001F00201CA2B006E00509EA8FED7AD6E91
:10128000050ECA5DF2E1CFC0CBF21B0ECC6F0001A0
:101290003BDF200E9EA8FED7AD6E0201CDD780A207
:1012A00032D00001CF518008D8A002D002012BD04B
:1012B000010ECF5FC80E0201DA6F000174DC210E4F
:1012C0000201D36F000113DDCFC0D3F210DD0201A4
:1012D000CA6BCA51000135EC01F00201CA2B006E45
:1012E00000509EA8FED7AD6E050ECA5DF2E1CFC0DC
:1012F000CBF21B0ECC6F000107DF200E9EA8FED79D
:10130000AD6E0201CCD7A96ACFC0A8FFA69CA69E4D
:10131000A684F2CF00F0F29E0F01550EA76EAA0E22
:10132000A76EA682A6B2FED7A6940050F2120001C4
:1013300015DDECEF24F00201E039F00B006E0F0E2A
:1013400081140010816E00008186030E006E002E55
:10135000FED781960001000C0F0E9314F009936ED6
:101360009392939493968184000081860000813843
:101370000F0B0201E06F81960000818600D000D043
:10138000000081380F0BDF6F81960F0E9314936E60
:10139000939293949396E039006EF00E00160050ED
:1013A000DF11016E0001D7EF09F08192D5D701C09E
:1013B000DFF2020101AE02D00001F8D7DDA1819277
:1013C000DDB181820000819400008196DE39DF6FFB
:1013D0000F0EDF17DFC2E0F20001ADDF0201DE51C8
:1013E0000F0BDF6FE06F0001A6DF000C0F0E9314F0
:1013F000936E9392939493968192819481960F0E1B
:101400000201DA6F0001D3EC05F0010E0201CA6F90
:10141000CA5103080DE3030EE06F00018CDF050ED7
:101420000201DA6F0001D3EC05F00201CA2BF0D7FC
:10143000020EE06F00017FDF0201CA6BCA51030890
:1014400013E3036ACA51F2CFCBF2F29E000102EC21
:1014500000F00201CBBFF28ECC6FDD6BDE6F0001BE
:10146000A4DF0201CA2BEAD700011EEF25F002011A
:10147000DB2D03D0800EDC6F11D0DB51020803E1BD
:10148000C00EDC6F0BD0DB51030803E1940EDC6F60
:1014900005D0DB51040802E1D40EDC6F010EDA5DE9
:1014A000DC27DD6BDCC2DEF200017FDF000C020115
:1014B000D9510C0A000105E0060A10E0020A16E004
:1014C0001CD00201DD6B010EDE6F00016EDF020E2B
:1014D0000201DA6F0001D3EC05F017D0010E020112
:1014E000DA6F020EDB6F0001C2DF0FD00201DD6B8D
:1014F000100EDE6F000159DF08D0010E0201DD6F12
:10150000D9C2DEF2000151DF00D0000CEE6BED6BB2
:10151000EC6BEB6B190E0201CA6FCA3D01D023D0F0
:1015200084A001D0FDD784B001D0FDD784A219D00A
:10153000036A026A016A010E006ECA51CB6F07E0AE
:10154000D8900036013602360336CB2FF9D700503B
:101550000001EB130150EC130250ED130350EE1396
:101560000201CA07DAD70001000C0201CB6B0B9411
:101570000001FA6BF96B190E0201CA6FCA3D01D066
:101580002BD0EEC003F0EDC002F0ECC001F0EBC0D8
:1015900000F0CA51CC6F07E0D8900332023201321A
:1015A0000032CC2FF9D700A014D0D890CB35036AE5
:1015B000F2CFCCF2F29E000142EC01F00900F5CF2F
:1015C00003F00201CCBFF28E0001F91B0350FA1B9D
:1015D0000201CB2BCA07D2D7030E0001FA17F9512B
:1015E000D80808E1FA51030805E10B84610EFC6F8D
:1015F0002CD02BD0F951D40808E1FA51030805E1A9
:101600000B84620EFC6F21D020D0F9515C0808E1F8
:10161000FA51020805E10B84630EFC6F16D015D059
:10162000F951CC0808E1FA51030805E10B84430E97
:10163000FC6F0BD00AD0F951580807E1FA510208A3
:1016400004E10B84640EFC6F00D0000CFB6B020104
:101650009E6B9D6B300E0001FC6F0B94EE6BED6B7F
:10166000EC6BEB6B53DF81DF010EEA6E1F0EE96E50
:10167000F2CFCAF2F29E000E64EC01F00A000900FB
:10168000F550EE6E0009FBE10201CABFF28E9B9598
:10169000000152EF25F00201D1BF11D00F0E006EF4
:1016A000D03900160A0E005C03E2300E002602D08C
:1016B000D151002600C0D9F20001F9DE02010F0E5F
:1016C000D0170A0ED05D02E2300E02D0D19FD15168
:1016D000D027D0C2D9F20001EADE000C0201D1BF4E
:1016E00011D00F0E006ED03900160A0E005C03E216
:1016F000300E002602D0D151002600C0D9F20001E0
:10170000E9DC02010F0ED0170A0ED05D02E2300EA6
:1017100002D0D19FD151D027D0C2D9F20001DADC5A
:10172000000C80A23AD00201C95100080BE2C9079F
:10173000C9C2CAF2CA1FCB6BCAC2CCF20001E7EC25
:1017400005F002010BB014D0120EDA6F020EDB6F3F
:1017500000018DDE560E0201D96F0001A8DEC9C25C
:10176000D0F2570E0201D16F000195DF16D00201B1
:101770000BA014D0420ED06F010ED16F00017EEC91
:1017800006F0560E0201D96F0001A4DCC9C2D0F2E6
:10179000570E0201D16F0001A1DF020180A03AD0F3
:1017A000C951FE080BE3C92BC9C2CAF2CA1FCB6BD1
:1017B000CAC2CCF20001E7EC05F002010BB014D074
:1017C000120EDA6F020EDB6F000151DE560E0201BF
:1017D000D96F00016CDEC9C2D0F2570E0201D16F81
:1017E000000159DF16D002010BA014D0420ED06FB9
:1017F000010ED16F00017EEC06F0560E0201D96F8A
:10180000000168DCC9C2D0F2570E0201D16F00019D
:1018100065DF020180A638D0C851000809E2C80778
:10182000010ECB6FC8C2CCF20001E7EC05F002015B
:101830000BB014D0120EDA6F020EDB6F000117DE50
:10184000540E0201D96F000132DEC8C2D0F2570E29
:101850000201D16F00011FDF16D002010BA014D0CE
:10186000420ED06F010ED16F00017EEC06F0540ED7
:101870000201D96F00012EDCC8C2D0F2570E02015E
:10188000D16F00012BDF020180A439D0C851FE08BE
:1018900009E3C82B010ECB6FC8C2CCF20001E7EC04
:1018A00005F002010BB014D0120EDA6F020EDB6FDE
:1018B0000001DDDD540E0201D96F0001F8DDC8C260
:1018C000D0F2570E0201D16F0001E5DE17D0020100
:1018D0000BA015D0420ED06F010ED16F00017EEC2F
:1018E00006F0540E0201D96F00016AEC08F0C8C27C
:1018F000D0F2570E0201D16F0001F0DE020180A884
:101900002AD0020EA96EC8C2A8FFA69CA69EA684D5
:10191000F2CF00F0F29E0F01550EA76EAA0EA76E31
:10192000A682A6B2FED7A6940050F212030EA96EAC
:10193000C9C2A8FFA69CA69EA684F2CF00F0F29E84
:10194000550EA76EAA0EA76EA682A6B2FED7A694C3
:101950000050F212020180A206D0140EDA6F0001CC
:10196000D3EC05F0020180A006D0140EDA6F00015E
:10197000D3EC05F0020180A606D0140EDA6F000148
:10198000D3EC05F0020180A406D0140EDA6F00013A
:10199000D3EC05F0020180A806D0140EDA6F000126
:1019A000D3EC05F00201000166EF25F0FB510408BD
:1019B000D8B4FB6BFB530BE1FC51610808E1010E4D
:1019C000FB6FF0C0F2F0EFC0F1F038D036D0FB2D55
:1019D0000BD0FC51620808E1020EFB6FF0C0F4F07E
:1019E000EFC0F3F02BD029D0FB5102080BE1FC51E2
:1019F000630808E1030EFB6FF0C0F6F0EFC0F5F0EE
:101A00001DD01BD0FB5102080BE1FC51430808E13B
:101A1000030EFB6FF0C0F6F0EFC0F5F00FD00DD065
:101A2000FB5103080AE1FC51640807E1040EFB6F57
:101A3000F0C0F8F0EFC0F7F001D0FB6B22EF22F01E
:101A40000201BCAF02D0BC6B06D0BCBF04D0BC51FD
:101A50003208D8A0BC6B0BB05FD00A0EDA6F010E53
:101A6000DB6F000104DD0201BCAF10D0200ED96F86
:101A700000011DDD200E0201D96F000118DD200ECE
:101A80000201D96F000113DD45D00201BCBF15D0A2
:101A9000BCBF03D0BC51050810E32A0ED96F00016A
:101AA00006DD2A0E0201D96F000101DD2A0E0201B6
:101AB000D96F0001FCDC2ED00201BCBF18D0BC5194
:101AC000050815E2BCBF03D0BC51140810E32A0E70
:101AD000D96F0001ECDC2A0E0201D96F0001E7DCAE
:101AE000200E0201D96F0001E2DC14D00201BCBF5C
:101AF00012D0BC5114080FE22A0ED96F0001D7DCB6
:101B0000200E0201D96F0001D2DC200E0201D96F34
:101B10000001CDDC020198D0360ED06FD16B0001F0
:101B20007EEC06F00201BCAF11D0CA6BCA510001B5
:101B3000E1EC04F00201CA2B006ED96F00016AECDF
:101B400008F0050E0201CA5DF1E17ED0BCBF16D0DF
:101B5000BCBF03D0BC510A0811E3CA6BCA510001D3
:101B6000ECEC04F00201CA2B006ED96F00016AECA4
:101B700008F0050E0201CA5DF1E166D0BCBF19D0C4
:101B8000BC510A0816E2BCBF03D0BC51140811E3D3
:101B9000CA6BCA510001F7EC04F00201CA2B006EB7
:101BA000D96F00016AEC08F0050E0201CA5DF1E18F
:101BB0004BD0BCBF19D0BC51140816E2BCBF03D037
:101BC000BC511E0811E3CA6BCA51000102EC05F0BA
:101BD0000201CA2B006ED96F00016AEC08F0050EF5
:101BE0000201CA5DF1E130D0BCBF19D0BC511E0862
:101BF00016E2BCBF03D0BC51280811E3CA6BCA511E
:101C000000010DEC05F00201CA2B006ED96F000136
:101C10006AEC08F0050E0201CA5DF1E115D0BCBF07
:101C200013D0BC51280810E2CA6BCA51000118EC4D
:101C300005F00201CA2B006ED96F00016AEC08F0B2
:101C4000050E0201CA5DF1E10001000CEACFD7F2F6
:101C5000E9CFD6F20201D039F009D26FD227E20FD4
:101C6000D36F320FD56FD0510F0BD327D327D52782
:101C7000E90FD46FD427D427CF390F0BD427D5271A
:101C8000D437D537D51FD537CF510F0BD527D237FE
:101C9000070ED16F0A0ED407D527FDE3D307D4274B
:101CA000FDE3D207D327FDE3D107D227FDE3020EE0
:101CB000EA6ED10EE96E070ED615D69DE926D50E31
:101CC000E95CD8B4D68DEF50006E08E1D6BD06D0E1
:101CD000D6B90CD0D6B702D0200E03D0D687D6996D
:101CE000300E002600509EA8FED7AD6EEE50D6AD49
:101CF000E6D70001000C8E0E006ED5C201F0D4C2F2
:101D000002F0036A015209E102C001F0026A080E02
:101D1000005E015202E1006A08D0D89001BE04D0F2
:101D2000023601360006F9D7019E000C800ED8A2BB
:101D300002D00201D71B0201DC6BDD6BD3C2DBF2E8
:101D4000D751DB1BD251D8B4DFD0DA6F006ED65139
:101D5000D8B4E3D0DA5FD8B483D03EE3D7C2E0F2A0
:101D6000E08FD8C2DFF2D9C2DEF2DD6BD890E0336B
:101D7000DF33DE33DD33DA2FF8D7DBAF03D0DC819E
:101D8000E0D0DC91DA91DC89020EEA6ED50EE96EC4
:101D9000EBD0DC99DBBF0AD0DAA113D0E033DF331C
:101DA000DE33DD33002AD8B4C7D00BD0E0BF0CD06F
:101DB000D890DD37DE37DF37E0370006D8B4BCD047
:101DC000F5D7DC8D6DD0DC9DD3C2DBF2D3AF02D072
:101DD000E08FABD0E09FA9D0D6C2DAF2D6C200F035
:101DE000D251DA5FD3C2E0F2E08FD4C2DFF2D5C2C3
:101DF000DEF2DD6BD890E033DF33DE33DD33DA2F14
:101E0000F8D7DBAF03D0DC839CD0DC93DA91DC8B9A
:101E1000020EEA6ED90EE96EA7D0DC9BDBBF0AD0BA
:101E2000DAA113D0E033DF33DE33DD33002AD8B458
:101E300083D00BD0E0BF0CD0D890DD37DE37DF3752
:101E4000E0370006D8B478D0F5D7DC8F29D0DC9FF6
:101E5000D7C2DBF2D7AF02D0E08F67D0E09F65D06A
:101E6000D7C2E0F2E08FD8C2DFF2D9C2DEF2DBAF38
:101E700004D0E09FDC8565D0DC95DD6BDA91020E45
:101E8000EA6ED50EE96E70D0DBBF1CD0D3C2DBF298
:101E9000DAA106D0E033DF33DE33DD33002A4CE055
:101EA000DDAF0BD0DE2B09E1DF2B07E1E02B05E1F5
:101EB000E033DF33DE33002A3FE0DCBD84D7DCBF14
:101EC000C6D71CD0800EE01BE0AF04D03AD0D7C2FA
:101ED000DBF20AD0D3C2DBF2E05306E1DF5304E1C8
:101EE000DE5302E1006A21D0E0BF08D0D890DD3790
:101EF000DE37DF37E037002EF7D71ED0DBAF02D05A
:101F0000E08F13D0E09F11D0D6C200F0D7C2E0F22C
:101F1000D8C2DFF2D9C2DEF208D0D2C200F0D3C2FA
:101F2000E0F2D4C2DFF2D5C2DEF2E0C201F0DFC2DD
:101F300002F0DEC203F034D0006A016A026A036A6A
:101F40002FD0DD6BDE1FDF1FE01FDD1FDD2B05E166
:101F5000DE2B03E1DF2B01E1E02BDCB112D7DCB398
:101F600054D7DCB589D7B3D7EF50DE2705E3DF2B95
:101F700003E1E02BD8B4DA81ED52EF50DF2703E321
:101F8000E02BD8B4DA81ED52EF50EFBE01D0800AD9
:101F9000E027D8B0DA81DCB9FCD6DCBB3ED774D7F9
:101FA0000001000C0201D651D8B4A5D0E26FDA517D
:101FB000D8B4A1D0E25F05E37F0EE227D8B09BD072
:101FC00006D0810EE25FD8A096D0D8B494D0E2C2F9
:101FD00000F0016A026A036AE16BD7C2E0F2E08FA7
:101FE000D8C2DFF2D9C2DEF2190EE26FDD51DE5F38
:101FF0000DE2010EDF5F0AE2E05F08E2E15F06E268
:10200000E12BE02BDF2BDD51DE2728D0DC51DF5F19
:1020100012E2010EE05F0FE2E15F0DE2E12BE02B47
:10202000DC51DF27DD51DE2719E3DF2B17E1E02B41
:1020300015E1E12B13D0DB518009E05F0EE2010EC8
:10204000E15F0BE2E12BDB518009E027DC51DF2768
:10205000E9E3E02BE7E1E12BE5D70380E22F01D0B4
:102060000BD0D890DE37DF37E037E137D890033632
:1020700002360136E337BAD7E3A106D0D890013251
:1020800002320332E33302D0000635E0E3BF1ED054
:10209000D890DE37DF37E037E137DD51DE5F07E22A
:1020A000010EDF5F04E2E05F02E2E15F1AE3DC5170
:1020B000DF5F05E2010EE05F02E2E15F12E3DB5168
:1020C0008009E05F03E2010EE15F0BE3032A09E10F
:1020D000022A07E1012A05E1002A0DE0013202325D
:1020E0000332D7C2E2F2DB51E21BE2AF02D0018E33
:1020F00006D0019E04D0006A016A026A036A0001E8
:10210000000C0201D651B608D66F036AD7C2DAF2C4
:10211000D78FD890D733D833D93303320232013234
:102120000032D62FF6D7DAAF0BD0001E011E021EEA
:10213000031E002AD8B4012AD8B4022AD8B4032A2C
:102140000001000C0201D451D8B471D0006ED851F6
:10215000D8B46DD0002604E3810E002668E204D0D6
:102160007F0E005E64E363E0D5C2DCF2D951DC1B74
:10217000D58FD98FD751DB03F4CFDEF2D651DA03F6
:10218000F4CF03F0F3CFDDF2DB03F350DE27F4509E
:10219000DD23000E0322D751DA03F350DE27F4507B
:1021A000DD23000E026A03220222D551DB03F35025
:1021B000DD27F4500322000E0222D551DA03F3503A
:1021C0000326F4500222000E016A0122D751D903DE
:1021D000F350DD27F4500322000E02220122D651D3
:1021E000D903F3500326F4500222000E0122D551E8
:1021F000D903F3500226F4500122002A01BE05D073
:10220000DD370336023601360006000EDDAF0AD098
:10221000032A02220122015005E1025003E103508A
:1022200001E1002ADCBF018EDCAF019E04D0006A10
:10223000016A026A036A0001000CB60E006E036AAE
:10224000026A016A0201D251D311D411D51102E1FF
:10225000006A0DD0D89001BE09D0D237D337D43719
:10226000D537033602360136002EF4D7019E000121
:1022700082EF17F00201D651D803F3CF01F0F4CF6B
:1022800000F0D903F3500026D751D803F3500020B3
:10229000026E0001000C0201D751D919800BDB6FCF
:1022A000D7AF05D0D61FD71FD62BD8B4D72BD9AFD1
:1022B00005D0D81FD91FD82BD8B4D92B016A026AF0
:1022C000006A036AD95102E1D85118E0100EDA6FA2
:1022D000D890D637D73700360336D951035C02E1A0
:1022E000D851005C07E3D851005ED8A00306D9514D
:1022F000035ED88001360236DA2FEAD7DBAF05D08D
:10230000011E021E012AD8B4022A000191EF11F029
:10231000CFC2D7F2CEC2D6F2D1C2D9F2D0C2D8F251
:10232000BAD702C0D3F201C0D2F2D1C2D7F2D0C222
:10233000D6F2D3C2D9F2D2C2D8F29CDF0150020148
:10234000CE5DD46F0250CF59D56FD2C200F0D3C248
:1023500001F0D4C202F0D5C203F000016AEF18F018
:10236000FE6BFD6B0101036B0B980B9A0B9C010E2E
:10237000EA6E1F0EE96EF2CFCEF2F29E000E000161
:1023800023EC05F00A000900F550EE6E0009FBE1B0
:102390000201CEBFF28E010EEA6E290EE96EF2CF77
:1023A000CEF2F29E000E000130EC05F00A000900AA
:1023B000F550EE6E0009FBE10201CEBFF28E010E78
:1023C000EA6E790EE96EF2CFCEF2F29E000E0001B7
:1023D00030EC05F00A000900F550EE6E0009FBE153
:1023E0000201CEBFF28E9B95A06B9F6BC56BC46B39
:1023F000C76BC66BBF6BBE6BC16BC06BC26BC36B75
:10240000010EDA6FDB6F000137EC0AF00201CE6BD0
:10241000CE51000159EC05F00201CE2B006ED96FB0
:10242000000157EC0AF0140E0201CE5DF1E1010E3D
:10243000DA6F020EDB6F000137EC0AF00201CE6B9F
:10244000CE51000159EC05F00201CE2B006ED96F80
:10245000000157EC0AF0140E0201CE5DF1E1010E0D
:10246000DA6F030EDB6F000137EC0AF00201CE6B6E
:10247000CE51000159EC05F00201CE2B006ED96F50
:10248000000157EC0AF0140E0201CE5DF1E1010EDD
:10249000DA6F040EDB6F000137EC0AF00201CE6B3D
:1024A000CE51000159EC05F00201CE2B006ED96F20
:1024B000000157EC0AF0140E0201CE5DF1E10001BB
:1024C000000CF2C0FEF0F1C0FDF0F4310201CF6F5C
:1024D0000001F3310201CE6FCF33CE33CF33CE3391
:1024E000CF33CE33CF33CE33070ECF17CE511F0BA2
:1024F0000101036F0353D8B405D303510A0816E151
:10250000010EEA6E040EE96EF2CFCEF2F29E000EDC
:10251000000171EC01F00A000900F550EE6E0009AF
:10252000FBE10201CEBFF28EECD2010103510C0897
:1025300016E1010EEA6E040EE96EF2CFCEF2F29EC3
:10254000000E000184EC01F00A000900F550EE6E67
:102550000009FBE10201CEBFF28ED3D2010103518B
:10256000170816E1010EEA6E040EE96EF2CFCEF204
:10257000F29E000E000197EC01F00A000900F550F0
:10258000EE6E0009FBE10201CEBFF28EBAD201016C
:1025900003510E0816E1010EEA6E040EE96EF2CF49
:1025A000CEF2F29E000E0001AAEC01F00A00090032
:1025B000F550EE6E0009FBE10201CEBFF28EA1D212
:1025C0000101032D16D0010EEA6E040EE96EF2CF62
:1025D000CEF2F29E000E0001BDEC01F00A000900EF
:1025E000F550EE6E0009FBE10201CEBFF28E89D2FA
:1025F00001010351020816E1010EEA6E040EE96EB4
:10260000F2CFCEF2F29E000E0001D0EC01F00A00F3
:102610000900F550EE6E0009FBE10201CEBFF28E1B
:1026200070D201010351030816E1010EEA6E040E97
:10263000E96EF2CFCEF2F29E000E0001E3EC01F063
:102640000A000900F550EE6E0009FBE10201CEBF61
:10265000F28E57D201010351040816E1010EEA6E11
:10266000040EE96EF2CFCEF2F29E000E0001F6ECFF
:1026700001F00A000900F550EE6E0009FBE10201CD
:10268000CEBFF28E3ED201010351050816E1010EC4
:10269000EA6E040EE96EF2CFCEF2F29E000E000159
:1026A00009EC02F00A000900F550EE6E0009FBE1AA
:1026B0000201CEBFF28E25D201010351060816E1B8
:1026C000010EEA6E040EE96EF2CFCEF2F29E000E1B
:1026D00000011CEC02F00A000900F550EE6E000942
:1026E000FBE10201CEBFF28E0CD2010103510708BB
:1026F00016E1010EEA6E040EE96EF2CFCEF2F29E02
:10270000000E00012FEC02F00A000900F550EE6EF9
:102710000009FBE10201CEBFF28EF3D101010351AA
:10272000080816E1010EEA6E040EE96EF2CFCEF251
:10273000F29E000E000142EC02F00A000900F55082
:10274000EE6E0009FBE10201CEBFF28EDAD101018B
:102750000351090816E1010EEA6E040EE96EF2CF8C
:10276000CEF2F29E000E000155EC02F00A000900C4
:10277000F550EE6E0009FBE10201CEBFF28EC1D131
:10278000010103510B0816E1010EEA6E040EE96E19
:10279000F2CFCEF2F29E000E000168EC02F00A00C9
:1027A0000900F550EE6E0009FBE10201CEBFF28E8A
:1027B000A8D1010103510D0816E1010EEA6E040EC5
:1027C000E96EF2CFCEF2F29E000E00017BEC02F039
:1027D0000A000900F550EE6E0009FBE10201CEBFD0
:1027E000F28E8FD1010103510F0816E1010EEA6E3E
:1027F000040EE96EF2CFCEF2F29E000E00018EECD6
:1028000002F00A000900F550EE6E0009FBE102013A
:10281000CEBFF28E76D101010351100816E1010EF0
:10282000EA6E040EE96EF2CFCEF2F29E000E0001C7
:10283000A1EC02F00A000900F550EE6E0009FBE180
:102840000201CEBFF28E5DD101010351110816E1E4
:10285000010EEA6E040EE96EF2CFCEF2F29E000E89
:102860000001B4EC02F00A000900F550EE6E000918
:10287000FBE10201CEBFF28E44D1010103511208E7
:1028800016E1010EEA6E040EE96EF2CFCEF2F29E70
:10289000000E0001C7EC02F00A000900F550EE6ED0
:1028A0000009FBE10201CEBFF28E2BD101010351E1
:1028B000130816E1010EEA6E040EE96EF2CFCEF2B5
:1028C000F29E000E0001DAEC02F00A000900F55059
:1028D000EE6E0009FBE10201CEBFF28E12D10101C2
:1028E0000351140816E1010EEA6E040EE96EF2CFF0
:1028F000CEF2F29E000E0001EDEC02F00A0009009B
:10290000F550EE6E0009FBE10201CEBFF28EF9D068
:1029100001010351150816E1010EEA6E040EE96E7D
:10292000F2CFCEF2F29E000E000100EC03F00A009E
:102930000900F550EE6E0009FBE10201CEBFF28EF8
:10294000E0D001010351160816E1010EEA6E040EF3
:10295000E96EF2CFCEF2F29E000E000113EC03F00E
:102960000A000900F550EE6E0009FBE10201CEBF3E
:10297000F28EC7D001010351180816E1010EEA6E6C
:10298000040EE96EF2CFCEF2F29E000E000126ECAC
:1029900003F00A000900F550EE6E0009FBE10201A8
:1029A000CEBFF28EAED001010351190816E1010E1F
:1029B000EA6E040EE96EF2CFCEF2F29E000E000136
:1029C00039EC03F00A000900F550EE6E0009FBE156
:1029D0000201CEBFF28E95D0010103511A0816E113
:1029E000010EEA6E040EE96EF2CFCEF2F29E000EF8
:1029F00000014CEC03F00A000900F550EE6E0009EE
:102A0000FBE10201CEBFF28E7CD0010103511B0815
:102A100016E1010EEA6E040EE96EF2CFCEF2F29EDE
:102A2000000E00015FEC03F00A000900F550EE6EA5
:102A30000009FBE10201CEBFF28E63D00101035118
:102A40001C0816E1010EEA6E040EE96EF2CFCEF21A
:102A5000F29E000E000172EC03F00A000900F5502E
:102A6000EE6E0009FBE10201CEBFF28E4AD00101F9
:102A700003511D0816E1010EEA6E040EE96EF2CF55
:102A8000CEF2F29E000E000185EC03F00A00090070
:102A9000F550EE6E0009FBE10201CEBFF28E31D09F
:102AA000010103511E0816E1010EEA6E040EE96EE3
:102AB000F2CFCEF2F29E000E000198EC03F00A0075
:102AC0000900F550EE6E0009FBE10201CEBFF28E67
:102AD00018D0010103511F0815E1010EEA6E040E22
:102AE000E96EF2CFCEF2F29E000E0001ABEC03F0E5
:102AF0000A000900F550EE6E0009FBE10201CEBFAD
:102B0000F28E0101F4C0CEF20201CE51F00B0101B0
:102B10001D6F0001F4B704D00A0E01011D1300015E
:102B2000F4A703D00B0E01011D1301011D510A086A
:102B300003E01D510B0832E10B960001F3B50B8643
:102B40000BA600D0F351030B0201CE6FCF6BD890D0
:102B5000CE35026ECF3502C01EF10101010E1E25D9
:102B6000036A1F0FE96E010E0320EA6E0001F7C031
:102B7000EFFF036A01011E511F0FE96E010E0320D2
:102B8000EA6E0201F8C0EFFF0B980001F4B50B8864
:102B90000B9AF3B90B8A6BEF1AF001011D512A0849
:102BA0007AE10001F3510F0B0201CE6FCF6BCE35EE
:102BB000026ECF35036E02360336FC0E021602C0DB
:102BC00028F101010B9E0001F3B90B8E0BBE31D031
:102BD000030E01012825036A290FE96E010E032067
:102BE000EA6E0001F7C0EFFF020E01012825036A1B
:102BF000290FE96E010E0320EA6E0201F8C0EFFF13
:102C0000010E01012825036A290FE96E010E032038
:102C1000EA6E0001F5C0EFFF036A01012851290F98
:102C2000E96E010E0320EA6E0201F6C0EFFF30D01C
:102C30000001030E01012825036A790FE96E010ED8
:102C40000320EA6E0001F7C0EFFF020E0101282504
:102C5000036A790FE96E010E0320EA6E0201F8C0E3
:102C6000EFFF010E01012825036A790FE96E010EBD
:102C70000320EA6E0001F5C0EFFF036A010128514D
:102C8000790FE96E010E0320EA6E0201F6C0EFFF34
:102C90006BEF1AF001011D514A08D8A467EF1AF032
:102CA00002019B95D8900001F6310201A06F00014E
:102CB000F53102019F6F0001F3A103D00201A08F43
:102CC0000001F3A300D0000E02019BB1010E000829
:102CD00024E2CE6BCE510001BEEC03F00201CE2BFC
:102CE000006E00509EA8FED7AD6E080ECE5DF2E1DC
:102CF000100EE96EA0C2D0F29FC2CFF2000126EC06
:102D00000EF0200E9EA8FED7AD6E0A0E9EA8FED72E
:102D1000AD6E0D0E9EA8FED7AD6E0001F551010BF4
:102D20000201CE6FCF6BCE35026ECF35036E023609
:102D300003360236033602360336F00E021602C0A0
:102D4000B2F2D16BB2C2D0F2B2BFD1070001F839F2
:102D50000201CE6F0F0ECE17CE510F0B006E036A1D
:102D60000050B225016ED151032201C0B2F2000120
:102D7000F8310201CF6F0001F7310201CE6FCF337E
:102D8000CE33CF33CE33CF33CE33CF33CE33CF3337
:102D9000CE33030ECF17CE513F0BB36F9B93000181
:102DA000F7AB03D002019B830001F7510F0B020127
:102DB000B16F9BB30BD0D890B131B227B2BF05D061
:102DC000B251170802E2180EB25F07D0D890B131A5
:102DD000B25FB2AF02D0180EB227A0C2D5F29FC226
:102DE000D4F200017BEC0EF0D88203C0D5F202C011
:102DF000D4F201C0D3F200C0D2F2CD0E0201D96FDD
:102E0000980ED86F6B0ED76F8C0ED66F000196ECB4
:102E10000EF000C0CEF201C0CFF202C0D0F203C06B
:102E2000D1F203C0D9F202C0D8F201C0D7F200C07B
:102E3000D6F20201DD6BA00EDC6F360EDB6F870E63
:102E4000DA6F0001D2EC0FF003C0D9F202C0D8F261
:102E500001C0D7F200C0D6F281EC10F001C0A2F29E
:102E600000C0A1F2A0C2D5F29FC2D4F27BEC0EF05A
:102E7000D88203C0D5F202C0D4F201C0D3F200C0A0
:102E8000D2F2660E0201D96FB00ED86F690ED76FFD
:102E90008C0ED66F000196EC0EF000C0CEF201C091
:102EA000CFF202C0D0F203C0D1F2A2C2D5F2A1C2C9
:102EB000D4F27BEC0EF003C0D7F202C0D6F201C010
:102EC000D5F200C0D4F20201DB6BA00EDA6F360E31
:102ED000D96F870ED86F0001A2EC10F003C0D9F2B1
:102EE00002C0D8F201C0D7F200C0D6F281EC10F0D7
:102EF00003C0D5F202C0D4F201C0D3F200C0D2F2B6
:102F00001DEF11F0D882D1C2D5F2D0C2D4F2CFC217
:102F1000D3F2CEC2D2F203C0D9F202C0D8F201C0BD
:102F2000D7F200C0D6F296EC0EF000C0D2F201C08B
:102F3000D3F202C0D4F203C0D5F203C0D9F202C06A
:102F4000D8F201C0D7F200C0D6F2010E0201DD6F47
:102F5000CD0EDC6F740EDB6F830EDA6F0001D2ECE6
:102F60000FF003C0D9F202C0D8F201C0D7F200C0FE
:102F7000D6F281EC10F001C0A4F200C0A3F26C0EF6
:102F800002019F5DCE6F3A0EA059CF6FA2C2D5F25B
:102F9000A1C2D4F200017BEC0EF003C0D7F202C054
:102FA000D6F201C0D5F200C0D4F20201DB6BA00E54
:102FB000DA6F360ED96F870ED86F0001A2EC10F0D1
:102FC00003C0D9F202C0D8F201C0D7F200C0D6F2D5
:102FD00081EC10F000500201CE5DD06F0150CF594E
:102FE000D16F000E0254D26F000E0354D36FA4C2EF
:102FF000D5F2A3C2D4F200017BEC0EF003C0D7F2ED
:1030000002C0D6F201C0D5F200C0D4F2010E020116
:10301000DB6FCD0EDA6F740ED96F830ED86F00019F
:10302000A2EC10F003C0D9F202C0D8F201C0D7F26E
:1030300000C0D6F281EC10F000500201D05DA56F07
:103040000150D159A66FA3510E0802E1A45305E027
:10305000A3510F0806E1A45304E1A86B010EA76F6A
:1030600002D0A86BA76BA751A125A96FA851A221D7
:10307000AA6F010EA35DCE6F000EA459CF6FA8C238
:10308000D7F2A7C2D6F2D96B0C0ED86F00013AEC7A
:1030900011F001500201CE5DAB6F0250CF59AC6F01
:1030A0006C0EA927070EAA23020E9F25CE6F000ED5
:1030B000A021CF6F350ECE5DAF6FD10ECF59B06F5F
:1030C000B0C2CFF2AFC2CEF2D16B070ED06F00010B
:1030D00088EF11F003C0CDF202C0CCF201C0CBF2F8
:1030E00000C0CAF2010E0201CC25016E000ECD21F6
:1030F00001C0ADF2AE6FAD2D17D0AE5315E1020E8B
:10310000EA6EB40EE96EF2CFCEF2F29E000E00012E
:10311000CEEC03F00A000900F550EE6E0009FBE169
:103120000201CEBFF28E9BD0AD51020817E1AE5323
:1031300015E1020EEA6EB40EE96EF2CFCEF2F29E07
:10314000000E0001D8EC03F00A000900F550EE6E05
:103150000009FBE10201CEBFF28E81D0AD51030820
:1031600017E1AE5315E1020EEA6EB40EE96EF2CF2E
:10317000CEF2F29E000E0001E2EC03F00A0009001C
:10318000F550EE6E0009FBE10201CEBFF28E67D072
:10319000AD51040817E1AE5315E1020EEA6EB40E0C
:1031A000E96EF2CFCEF2F29E000E0001ECEC03F0DD
:1031B0000A000900F550EE6E0009FBE10201CEBFE6
:1031C000F28E4DD0AD51050817E1AE5315E1020E58
:1031D000EA6EB40EE96EF2CFCEF2F29E000E00015E
:1031E000F6EC03F00A000900F550EE6E0009FBE171
:1031F0000201CEBFF28E33D0AD51060817E1AE53B7
:1032000015E1020EEA6EB40EE96EF2CFCEF2F29E36
:10321000000E000100EC04F00A000900F550EE6E0B
:103220000009FBE10201CEBFF28E19D0AD510708B3
:1032300016E1AE5314E1020EEA6EB40EE96EF2CF5F
:10324000CEF2F29E000E00010AEC04F00A00090022
:10325000F550EE6E0009FBE10201CEBFF28EAB2D00
:1032600017D0AC5315E1020EEA6EB80EE96EF2CF3C
:10327000CEF2F29E000E000114EC04F00A000900E8
:10328000F550EE6E0009FBE10201CEBFF28E1DD1BA
:10329000AB51020817E1AC5315E1020EEA6EB80E0D
:1032A000E96EF2CFCEF2F29E000E00011EEC04F0A9
:1032B0000A000900F550EE6E0009FBE10201CEBFE5
:1032C000F28E03D1AB51030817E1AC5315E1020EA6
:1032D000EA6EB80EE96EF2CFCEF2F29E000E000159
:1032E00028EC04F00A000900F550EE6E0009FBE13D
:1032F0000201CEBFF28EE9D0AB51040817E1AC5306
:1033000015E1020EEA6EB80EE96EF2CFCEF2F29E31
:10331000000E000132EC04F00A000900F550EE6ED8
:103320000009FBE10201CEBFF28ECFD0AB51050800
:1033300017E1AC5315E1020EEA6EB80EE96EF2CF5A
:10334000CEF2F29E000E00013CEC04F00A000900EF
:10335000F550EE6E0009FBE10201CEBFF28EB5D052
:10336000AB51060817E1AC5315E1020EEA6EB80E38
:10337000E96EF2CFCEF2F29E000E000146EC04F0B0
:103380000A000900F550EE6E0009FBE10201CEBF14
:10339000F28E9BD0AB51070817E1AC5315E1020E3A
:1033A000EA6EB80EE96EF2CFCEF2F29E000E000188
:1033B00050EC04F00A000900F550EE6E0009FBE144
:1033C0000201CEBFF28E81D0AB51080817E1AC5399
:1033D00015E1020EEA6EB80EE96EF2CFCEF2F29E61
:1033E000000E00015AEC04F00A000900F550EE6EE0
:1033F0000009FBE10201CEBFF28E67D0AB51090894
:1034000017E1AC5315E1020EEA6EB80EE96EF2CF89
:10341000CEF2F29E000E000164EC04F00A000900F6
:10342000F550EE6E0009FBE10201CEBFF28E4DD0E9
:10343000AB510A0817E1AC5315E1020EEA6EB80E63
:10344000E96EF2CFCEF2F29E000E00016EEC04F0B7
:103450000A000900F550EE6E0009FBE10201CEBF43
:10346000F28E33D0AB510B0817E1AC5315E1020ECD
:10347000EA6EB80EE96EF2CFCEF2F29E000E0001B7
:1034800078EC04F00A000900F550EE6E0009FBE14B
:103490000201CEBFF28E19D0AB510C0816E1AC532D
:1034A00014E1020EEA6EB80EE96EF2CFCEF2F29E91
:1034B000000E000182EC04F00A000900F550EE6EE7
:1034C0000009FBE10201CEBFF28E05D001011D51C2
:1034D0008A0801E10B8C0201AA5106080DE2FF0ADD
:1034E00003E1A951D50808E2AA51080805E303E160
:1034F000A9510208D8B09B8500C102F1FFC001F1BB
:10350000FEC000F1FDC0FFF0010101510001FF5DAF
:1035100005E101010251005D1FE00001FD5302E1E0
:10352000FE5319E00101036B140E02019C6FCE6B78
:10353000CE5100018CEC04F00201CE2B006E005045
:103540009EA8FED7AD6E140ECE5DF2E10001B0EC88
:1035500011F00B980B9A0101000135EF22F0EACF30
:10356000D8F2E9CFD7F20201D139F009D36FD327CE
:10357000E20FD46F320FD66FD1510F0BD427D4275F
:10358000D627E90FD56FD527D527D0390F0BD527EB
:10359000D627D537D637D61FD637D0510F0BD627DB
:1035A000D337070ED26F0A0ED507D627FDE3D4070F
:1035B000D527FDE3D307D427FDE3D207D327FDE3C7
:1035C000020EEA6ED20EE96E070ED715D79DE926D8
:1035D000D60EE95CD8B4D78DEF50006E08E1D7BDA8
:1035E00006D0D7B916D0D7B702D0200E03D0D787D0
:1035F000D799300E0026EACFD1F2E9CFD0F200C041
:10360000D9F2000157EC0AF0D1C2EAFFD0C2E9FFBB
:103610000201EE50D7ADDCD70001000C0150D0C242
:10362000D2F2640E0201D36F00016EEC08F000C00C
:10363000D0F20150300E08E10201D1A310D0D1B771
:103640000ED0D1B9200E04D00201D197D199D181E9
:10365000012601C0D9F2000157EC0AF00201D0C2E4
:10366000D2F20A0ED36F00016EEC08F000C0D0F267
:103670000150300E08E10201D1B70BD0D1A109D021
:10368000D1B9200E0001012601C0D9F257EC0AF091
:103690000201300ED027D0C2D9F2000157EC0AF057
:1036A000000CD1C2D3F2D0C2D2F2D3C203F00201D5
:1036B000D2C2E9FFD3C2EAFFEF5206E0D22BD8B460
:1036C000D32B0001F2D70201D051D25D006ED1514F
:1036D000D359036E00C001F0026E0001000CD1C28C
:1036E000D6F2D0C2D5F20201D45324E0D3C203F003
:1036F000D2C2E9FFD3C2EAFFEF521CE0D6C203F008
:10370000D551D52BD8B4D62BD76F03C0D8F2D3C29E
:1037100003F0D251D22BD8B4D32BE96E03C0EAFF09
:10372000EFCFD9F2D8C2EAFFD7C2E9FFD9C2EFFF83
:10373000D407DAD7D4530CE0D6C203F0D551D52B39
:10374000D8B4D62BE96E03C0EAFFEF6AD407F2D7EC
:10375000D0C201F0D1C202F00001000C010E020142
:10376000DA6FDB6F000137EC0AF0010EEA6E1F0E14
:10377000E96E000EEF1010E0EACFD1F2E9CFD0F2FF
:10378000EFCFD9F257EC0AF0D1C2EAFFD0C2E9FF7D
:10379000E92AD8B4EA2AEDD70E0E0201DA6F010E3B
:1037A000DB6F000137EC0AF0FD5302E1FE5311E03C
:1037B000FEC0D0F2570E0201D16F00014BEC0BF0AE
:1037C000FDC0D0F2570E0201D16F00014BEC0BF09F
:1037D00011D00201D06BD0510001C6EC04F00201FF
:1037E000D02B006ED96F000157EC0AF0040E0201D5
:1037F000D05DF1E1130E0201DA6F010EDB6F000103
:1038000037EC0AF00BAC0DD0540E0201D96F000159
:1038100057EC0AF04D0E0201D96F000157EC0AF087
:103820002CD00BBC2AD00BA81CD00BAA0DD0540E48
:103830000201D96F000157EC0AF0410E0201D96F65
:10384000000157EC0AF00CD0540E0201D96F0001B0
:1038500057EC0AF0500E0201D96F000157EC0AF044
:103860000CD0200E0201D96F000157EC0AF0200E97
:103870000201D96F000157EC0AF002019BA554D058
:10388000010EDA6F020EDB6F000137EC0AF0030E57
:10389000E96EA6C2D1F2A5C2D0F261DE200E02010D
:1038A000D96F000157EC0AF0020EEA6EB80EE96E0D
:1038B000000EEF1010E0EACFD1F2E9CFD0F2EFCF57
:1038C000D9F257EC0AF0D1C2EAFFD0C2E9FFE92AE7
:1038D000D8B4EA2AEDD7200E0201D96F000157ECC7
:1038E0000AF0010EE96EAAC2D1F2A9C2D0F237DE07
:1038F000200E0201D96F000157EC0AF0B2C2D0F2DB
:10390000110E0201D16F000189DE3A0E0201D96F5A
:10391000000157EC0AF0B3C2D0F2010E0201D16FE0
:1039200000017CDE02019B95CE6BCE513F0820E06A
:10393000036ACE51290FE96E010E0320EA6EEF50A3
:10394000F00B14E1CEC2CFF2CF5140080BE0036A76
:10395000CF51290FE96E010E0320EA6E200EEF6EA3
:10396000CF2BF2D70101696B03D00201CE2BDDD73B
:103970000201CE6BCE513F0820E0036ACE51790F91
:10398000E96E010E0320EA6EEF50F00B14E1CEC297
:10399000CFF2CF5140080BE0036ACF51790FE96EA7
:1039A000010E0320EA6E200EEF6ECF2BF2D701013D
:1039B000B96B03D00201CE2BDDD70201C55303E161
:1039C000C4512C0843E2BF5303E1BE5101083DE25C
:1039D000BF6BBE6B010ED16F290ED06F000161DE8F
:1039E00001C0CAF20201CC6BCA51CC5D1AE0036A75
:1039F000CC51C90F016E010E032203C0D1F2CC518C
:103A0000C225036A290FE96E010E0320EA6EEFCF8B
:103A1000D3F2D1C2EAFF01C0E9FFD3C2EFFFCC2B42
:103A2000E3D7020ED16F690ED06F010ED36FC90EAE
:103A3000D26F140ED46F000152DE0201C22BCA51A4
:103A4000C25D03E1C26BC56BC46B10D0C42BD8B48C
:103A5000C52B020ED16F690ED06F010ED36F290EE8
:103A6000D26F140ED46F00013ADE0201BE2BD8B41F
:103A7000BF2B010EDA6F030EDB6F000137EC0AF08B
:103A8000020EEA6E690EE96E000EEF1010E0EACF4A
:103A9000D1F2E9CFD0F2EFCFD9F257EC0AF0D1C290
:103AA000EAFFD0C2E9FFE92AD8B4EA2AEDD7020139
:103AB000C75303E1C6512C0843E2C15303E1C0518F
:103AC00001083DE2C16BC06B010ED16F790ED06F62
:103AD0000001E7DD01C0CBF20201CD6BCB51CD5D22
:103AE0001AE0036ACD51190F016E020E032203C0C2
:103AF000D1F2CD51C325036A790FE96E010E03207F
:103B0000EA6EEFCFD3F2D1C2EAFF01C0E9FFD3C220
:103B1000EFFFCD2BE3D7020ED16F820ED06F020ED6
:103B2000D36F190ED26F140ED46F0001D8DD0201CD
:103B3000C32BCB51C35D03E1C36BC76BC66B10D006
:103B4000C62BD8B4C72B020ED16F820ED06F010ED8
:103B5000D36F790ED26F140ED46F0001C0DD020155
:103B6000C02BD8B4C12B010EDA6F040EDB6F00013D
:103B700037EC0AF0020EEA6E820EE96E000EEF10CC
:103B800010E0EACFD1F2E9CFD0F2EFCFD9F257EC83
:103B90000AF0D1C2EAFFD0C2E9FFE92AD8B4EA2A82
:103BA000EDD7000C0201CBBF10D00F0E006ECA394A
:103BB00000160A0E005C03E2300E002602D0CB5144
:103BC000002600509EA8FED7AD6E0F0ECA170A0E33
:103BD000CA5D02E2300E02D0CB9FCB51CA27CA5138
:103BE0009EA8FED7AD6E0001000C010EEA6E1F0EFE
:103BF000E96E000EEF1008E0EF509EA8FED7AD6E04
:103C0000E92AD8B4EA2AF5D7200E9EA8FED7AD6ED1
:103C1000200E9EA8FED7AD6EFEC0CAF2570E02015E
:103C2000CB6F0001BFDFFDC0CAF2570E0201CB6FA0
:103C30000001B8DF200E9EA8FED7AD6E200E9EA814
:103C4000FED7AD6E200E9EA8FED7AD6E03C1CBF29F
:103C50001B0E0201CC6F000184EC08F0200E9EA820
:103C6000FED7AD6E0BA812D00201CA6BCA5100017B
:103C70009FEC04F00201CA2B006E00509EA8FED7F4
:103C8000AD6E040ECA5DF2E10ED00001200E9EA8BA
:103C9000FED7AD6E200E9EA8FED7AD6E200E9EA85C
:103CA000FED7AD6E02010BAA0DD0540E9EA8FED712
:103CB000AD6E410E9EA8FED7AD6E200E9EA8FED71B
:103CC000AD6E0CD0200E9EA8FED7AD6E200E9EA825
:103CD000FED7AD6E200E9EA8FED7AD6E9BA55BD025
:103CE000B2C2CBF2110ECC6F000184EC08F03A0E98
:103CF0009EA8FED7AD6EB3C2CBF2010E0201CC6F0F
:103D0000000184EC08F0200E9EA8FED7AD6E020ED6
:103D1000EA6EB40EE96E000EEF1008E0EF509EA8B8
:103D2000FED7AD6EE92AD8B4EA2AF5D7200E9EA8B0
:103D3000FED7AD6E020EEA6EB80EE96E000EEF1001
:103D400008E0EF509EA8FED7AD6EE92AD8B4EA2A63
:103D5000F5D7200E9EA8FED7AD6E0B0EE96EA6C25B
:103D6000D0F2A5C2CFF226EC0EF02C0E9EA8FED704
:103D7000AD6E200E9EA8FED7AD6E010EE96EAAC2F2
:103D8000D0F2A9C2CFF226EC0EF0200E9EA8FED7EC
:103D9000AD6E11D00201CA6BCA510001AAEC04F049
:103DA0000201CA2B006E00509EA8FED7AD6E100E09
:103DB000CA5DF2E10001200E9EA8FED7AD6E0A0E8C
:103DC0009EA8FED7AD6E0D0E9EA8FED7AD6E010E5D
:103DD000EA6E290EE96E000EEF1008E0EF509EA883
:103DE000FED7AD6EE92AD8B4EA2AF5D7200E9EA8F0
:103DF000FED7AD6E0A0E9EA8FED7AD6E0D0E9EA824
:103E0000FED7AD6E010EEA6E790EE96E000EEF1070
:103E100008E0EF509EA8FED7AD6EE92AD8B4EA2A92
:103E2000F5D70201CA6BCA510001BBEC04F00201D4
:103E3000CA2B006E00509EA8FED7AD6E040ECA5D60
:103E4000F2E10001000C0150D0C2D2F2640E020176
:103E5000D36F00016EEC08F000C0D0F20150300EBC
:103E600008E10201D1A310D0D1B70ED0D1B9200EF4
:103E700004D00201D197D199D181012601C0D9F294
:103E800000016AEC08F00201D0C2D2F20A0ED36F30
:103E900000016EEC08F000C0D0F20150300E08E1D5
:103EA0000201D1B70BD0D1A109D0D1B9200E0001A8
:103EB000012601C0D9F26AEC08F00201300ED027C9
:103EC000D0C2D9F200016AEC08F0000CEACFD8F2B7
:103ED000E9CFD7F20201D139F009D36FD327E20F2E
:103EE000D46F320FD66FD1510F0BD427D427D627DA
:103EF000E90FD56FD527D527D0390F0BD527D62772
:103F0000D537D637D61FD637D0510F0BD627D33754
:103F1000070ED26F0A0ED507D627FDE3D407D527A3
:103F2000FDE3D307D427FDE3D207D327FDE3020E39
:103F3000EA6ED20EE96E070ED715D79DE926D60E8A
:103F4000E95CD8B4D78DEF50006E08E1D7BD06D03C
:103F5000D7B916D0D7B702D0200E03D0D787D799BC
:103F6000300E0026EACFD1F2E9CFD0F200C0D9F26C
:103F700000016AEC08F0D1C2EAFFD0C2E9FF0201F9
:103F8000EE50D7ADDCD70001000C0201D06BD16B35
:103F900000017EEC06F0010EEA6E1F0EE96E000EC7
:103FA000EF1010E0EACFD1F2E9CFD0F2EFCFD9F2A3
:103FB0006AEC08F0D1C2EAFFD0C2E9FFE92AD8B41E
:103FC000EA2AEDD7FD5302E1FE5318E0240E020168
:103FD000D06F010ED16F00017EEC06F0FEC0D0F272
:103FE000570E0201D16F00016EEC0BF0FDC0D0F254
:103FF000570E0201D16F00016EEC0BF00201D06B85
:10400000020ED16F00017EEC06F00BA813D0540E07
:104010000201D96F00016AEC08F0500E0201D96F5D
:1040200000016AEC08F0200E0201D96F00016AEC71
:1040300008F012D0200E0201D96F00016AEC08F0DE
:10404000200E0201D96F00016AEC08F0200E020177
:10405000D96F00016AEC08F00BAA0DD0540E0201D2
:10406000D96F00016AEC08F0410E0201D96F00011E
:104070006AEC08F00CD0200E0201D96F00016AEC46
:1040800008F0200E0201D96F00016AEC08F0360E2C
:104090000201D06F020ED16F00017EEC06F002012A
:1040A0009BA55AD0B2C2D0F2110ED16F0001CBDE67
:1040B0003A0E0201D96F00016AEC08F0B3C2D0F2E7
:1040C000010E0201D16F0001BEDE200E0201D96F88
:1040D00000016AEC08F0120E0201D06F030ED16FDE
:1040E00000017EEC06F0020EEA6EB80EE96E000EDC
:1040F000EF1010E0EACFD1F2E9CFD0F2EFCFD9F252
:104100006AEC08F0D1C2EAFFD0C2E9FFE92AD8B4CC
:10411000EA2AEDD7200E0201D96F00016AEC08F0FF
:104120000B0EE96EA6C2D1F2A5C2D0F2CFDE200EF0
:104130000201D96F00016AEC08F0010EE96EAAC213
:10414000D1F2A9C2D0F2C2DE200E0201D96F000165
:104150006AEC08F012D00201D06BD0510001D1EC12
:1041600004F00201D02B006ED96F00016AEC08F058
:104170000F0E0201D05DF1E100010201CE6BCE51C4
:104180003F0820E0036ACE51290FE96E010E03209B
:10419000EA6EEF50F00B14E1CEC2CFF2CF514008DF
:1041A0000BE0036ACF51290FE96E010E0320EA6E7E
:1041B000200EEF6ECF2BF2D70101696B03D0020105
:1041C000CE2BDDD70201CE6BCE513F0820E0036A33
:1041D000CE51790FE96E010E0320EA6EEF50F00B1D
:1041E00014E1CEC2CFF2CF5140080BE0036ACF51A9
:1041F000790FE96E010E0320EA6E200EEF6ECF2BD1
:10420000F2D70101B96B03D00201CE2BDDD7020139
:10421000C55303E1C4512C0845E2BF5303E1BE512D
:1042200001083FE2BF6BBE6B010ED16F290ED06F4C
:10423000000151EC1BF001C0CAF20201CC6BCA5163
:10424000CC5D1AE0036ACC51C90F016E010E032246
:1042500003C0D1F2CC51C225036A290FE96E010EC9
:104260000320EA6EEFCFD3F2D1C2EAFF01C0E9FF2B
:10427000D3C2EFFFCC2BE3D7020ED16F690ED06F04
:10428000010ED36FC90ED26F0E0ED46F00016FEC0A
:104290001BF00201C22BCA51C25D03E1C26BC56BA8
:1042A000C46B11D0C42BD8B4C52B020ED16F690ECC
:1042B000D06F010ED36F290ED26F0E0ED46F000196
:1042C0006FEC1BF00201BE2BD8B4BF2BD06B040ED9
:1042D000D16F00017EEC06F0020EEA6E690EE96E07
:1042E000000EEF1010E0EACFD1F2E9CFD0F2EFCF1D
:1042F000D9F26AEC08F0D1C2EAFFD0C2E9FFE92A9C
:10430000D8B4EA2AEDD70201C75303E1C6512C08FD
:1043100045E2C15303E1C05101083FE2C16BC06BEC
:10432000010ED16F790ED06F000151EC1BF001C06E
:10433000CBF20201CD6BCB51CD5D1AE0036ACD51BA
:10434000190F016E020E032203C0D1F2CD51C32515
:10435000036A790FE96E010E0320EA6EEFCFD3F204
:10436000D1C2EAFF01C0E9FFD3C2EFFFCD2BE3D7F3
:10437000020ED16F820ED06F020ED36F190ED26F64
:104380000E0ED46F00016FEC1BF00201C32BCB515A
:10439000C35D03E1C36BC76BC66B11D0C62BD8B42A
:1043A000C72B020ED16F820ED06F010ED36F790E24
:1043B000D26F0E0ED46F00016FEC1BF00201C02B08
:1043C000D8B4C12BD06B050ED16F00017EEC06F086
:1043D000020EEA6E820EE96E000EEF1010E0EACFD8
:1043E000D1F2E9CFD0F2EFCFD9F26AEC08F0D1C226
:1043F000EAFFD0C2E9FFE92AD8B4EA2AEDD7000CD7
:10440000D890EB37EC37ED37EE37030EEE1784A07C
:1044100001D0FDD784B001D0FDD784B2EB8193EFFA
:1044200022F00BA44CD0EE31026EED31016EEC3176
:10443000006E02320132003200C0EFF001C0F0F035
:10444000D6EF0CF0FB51040835E102019C2BBD2B8B
:10445000BC2BBD51640806E2000120EC0DF0320EC9
:104460000201BD6F000161EF12F00BB012D002012A
:104470009C5100080DE20001AEEC1BF002019BA173
:1044800004D00001F5EC1DF002019C6B9E6B9D6B4E
:1044900010D002019C5100080CE2000176DD0201FF
:1044A0009BA104D00001F5EC1DF002019C6B9E6BFA
:1044B0009D6B000186EC0AF0B5EC0AF0B2D70BB4A4
:1044C00035D002019D2BD8B49E2BBD2BBC07BD530C
:1044D00006E1000120EC0DF0320E0201BD6F0BB0C1
:1044E00011D09E5112080DE2FF0A03E19D51870889
:1044F00008E20001B0EC11F0AEEC1BF002019E6B83
:104500009D6B0FD09E5100080CE2FF0A03E19D5104
:10451000F30807E20001B0EC11F037DD02019E6BF9
:104520009D6B00016DD7B5EC0AF0C9D767EF25F098
:10453000F86AD09EFE0E006E060E016E020EE96E47
:10454000000EEA6EEE6A002EFDD7012EFBD7EA6A56
:10455000E96A0A0EAF6EA60EAC6E900EAB6EC1800D
:10456000C182C184C196056A066A1E0E0C6E210EB8
:104570000D6E610E0E6E210E0F6E120E106E3C0E41
:10458000116E410E126E400E136E210E146E7C0ED3
:10459000156E380E166E540E176E560E186E550E9A
:1045A000196E180E1A6E200E1B6E550E1C6E1D6EA7
:1045B0001E6E780E1F6E200E206E550E216E540E4C
:1045C000226E550E236E780E246E200E256E550E2B
:1045D000266E560E276E540E286E780E296E200E0B
:1045E0002A6E540E2B6E550E2C6E540E2D6E780EB8
:1045F0002E6E1C0E2F6E220E306E620E316E220E4B
:10460000326E100E336E380E346E550E356E366EB9
:10461000376E180E386E380E396E550E3A6E540ECF
:104620003B6E550E3C6E180E3D6E380E3E6E540EAF
:104630003F6E550E406E560E416E180E426E436A26
:10464000450E446E7C0E456E410E466E476A486AC2
:10465000450E496E7D0E4A6E410E4B6E4C6A4D6A98
:10466000450E4E6E7E0E4F6E400E506E516A780EA5
:10467000526E150E536E140E546E150E556E780E46
:10468000566E576E140E586E150E596E140E5A6EE5
:10469000780E5B6E7C0E5C6E540E5D6E560E5E6E1A
:1046A000550E5F6E440E606E240E616E540E626E87
:1046B000780E636E540E646E480E656E7E0E666EE6
:1046C000090E676E7E0E686E490E696E6A6E380E50
:1046D0006B6E450E6C6E6D6E6E6E380E6F6E706E1C
:1046E000450E716E440E726E450E736E380E746E0A
:1046F000756E450E766E460E776E440E786E380EE9
:10470000796E3C0E7A6E410E7B6E7C6E210E7D6E54
:104710007C0E7E6E3C0E7F6E410E806F420E816F6E
:10472000200E826F7C0E836F0C0E846F510E856F8E
:10473000500E866F510E876F3C0E886F380E896F52
:10474000450E8A6F440E8B6F450E8C6F380E8D6F41
:104750003C0E8E6F410E8F6F400E906F410E916F29
:104760003C0E926F936B946B956B966B976B200ED0
:10477000986F480E996F3E0E9A6F490E9B6F620EAE
:104780009C6F9D6B9E6B9F6BA06BA16BA26BA36BD1
:10479000A46BA56BA66B400EA76F680EA86F3E0EAC
:1047A000A96F090EAA6F020EAB6F200EAC6F540EEC
:1047B000AD6F560EAE6F550EAF6F780EB06FB16B1A
:1047C000440EB26F7E0EB36F410EB46FB56B380EF0
:1047D000B66F440EB76F460EB86F450EB96F380E00
:1047E000BA6F3C0EBB6F400EBC6F420EBD6F210E08
:1047F000BE6F7C0EBF6FC06F090EC16F050EC26F1A
:10480000C36F780EC46F7C0EC56F090EC66F110E94
:10481000C76F210EC86F7C0EC96F7E0ECA6F250E42
:10482000CB6FCC6F260ECD6F180ECE6FC290C180AD
:10483000C182C184C1961F0E926E000E936E900EBF
:10484000946EC10E956E968096829684828482863E
:1048500082928290F2CFCAF2F29E020EA96EA69CBC
:10486000A69EA680A8500201CABFF28EC86FC83D9E
:1048700002D0800EC86F010ECB6FC8C2CCF200010F
:10488000E7EC05F0F2CFCAF2F29E030EA96EA69CE9
:10489000A69EA680A8500201CABFF28EC96FC93D6C
:1048A00002D0020EC96FC9C2CAF2CA1FCB6BCAC2FC
:1048B000CCF20001E7EC05F00201CA6BCA5100011D
:1048C0006CEC05F00201CA2B006E00509EA8FED7CA
:1048D000AD6E140ECA5DF2E180A617D00B90040EE7
:1048E000A96EA86AA69CA69EA684F2CF00F0F29EAE
:1048F0000F01550EA76EAA0EA76EA682A6B2FED70E
:10490000A6940050F21219D0020180A417D00B8097
:10491000040EA96E010EA86EA69CA69EA684F2CFD8
:1049200000F0F29E0F01550EA76EAA0EA76EA6828A
:10493000A6B2FED7A6940050F212020180A601D0C2
:10494000FDD780A401D0FDD7F2CFCAF2F29E040EAB
:10495000A96EA69CA69EA680A850CABFF28EFF088C
:1049600017E10B90040EA96EA86AA69CA69EA684C9
:10497000F250006EF29E0F01550EA76EAA0EA76EA2
:10498000A682A6B2FED7A6940050F2121ED0020153
:10499000F2CFCAF2F29E040EA96EA69CA69EA68035
:1049A000A850CABFF28E000A02E10B900ED0F2CFDF
:1049B000CAF2F29E040EA96EA69CA69EA680A850DE
:1049C000CABFF28E010801E10B8000013CEF06F046
:1049D000AEEC06F0C3EF08F00201D06B040ED16F0D
:1049E00000017EEC06F00201CA6BCA5100017FECA7
:1049F00005F00201CA2B006ED96F00016AEC08F0C5
:104A00000E0E0201CA5DF1E1D06B050ED16F0001FF
:104A10007EEC06F00201CA6BCA5100018FEC05F072
:104A20000201CA2B006ED96F00016AEC08F00E0E6D
:104A30000201CA5DF1E10001F6EF09F0010E020189
:104A4000DA6F030EDB6F000137EC0AF00201CA6B6C
:104A5000CA5100019FEC05F00201CA2B006ED96F0C
:104A6000000157EC0AF0140E0201CA5DF1E1010EDB
:104A7000DA6F040EDB6F000137EC0AF00201CA6B3B
:104A8000CA510001B2EC05F00201CA2B006ED96FC9
:104A9000000157EC0AF0140E0201CA5DF1E10001B9
:104AA00026EF0BF00201CA6BCA510001C5EC05F0FC
:104AB0000201CA2B006E00509EA8FED7AD6E0A0EF2
:104AC000CA5DF2E19B81000191EF0BF0AAD4FCD703
:024AD0000300E1
:020000040030CA
:0E00000000220C0E000180000FC00FE00F4028
:00000001FF
